:020000040000FA
:100000000C280000000000008B018316C930850019
:100010008312ED3085000B288316DF308100FF301E
:10002000850003308E0000308F00013096002030B4
:10003000990000309F00831200308100203084003E
:100040000030850004308A0008308B0000309000BA
:10005000133098000730990000309F00031A3F28A2
:10006000031618108316C930850083123E308500B0
:100070003230A800032108308B00630000000B1011
:10008000181464003230A80005184228A80B442830
:100090000B101930A8000321A901AA01AB01FF3000
:1000A000A700A600063021020318A1010630230292
:1000B0000318A30121080024A500A50E230800248D
:1000C000A504622827088316850083122608850068
:1000D000FF30A700A600251E7128A71027122612A0
:1000E00074280000000000008500251C7B282711D3
:1000F000A712A6127E280000000000002708831621
:100100008500831226088500800AA20A00000000EC
:10011000FF30A700A600A51E9128A71227122612BD
:100120009428000000000000A51C9A282711A710A1
:10013000A6109D28000000000000850027088316F7
:100140008500831226088500840A840A04110000B1
:10015000FF30A700A600251FB1282712A710A61060
:10016000B428000000000000251DBA28A71227119E
:100170002611BD2800000000000085002708831616
:10018000850083122608850032300B18A9000B1059
:10019000FF30A700A600A51FD1282712A712A6127C
:1001A000D428000000000000A51DDA28A7102711A0
:1001B0002611DD2800000000000085002908031931
:1001C0006228AA070F302A02031C6228AA01013004
:1001D000A90303191930A80003212B18A50EF0302C
:1001E000A5050008FE24840A8007063000020318D3
:1001F000800000080024A50484032B18A50E0130FC
:10020000AB06640062280B088316051083120514E0
:100210000510A80B072983160514831285088B0087
:020220000800D4
:1008000007390A108207083404340C3405340D34D7
:0608100007340F34003430
:0409FC000A14820750
:100A0000023404340134033405340534043403342B
:100A1000023404340334043404340234013403341F
:100A20000434013404340434043405340534023409
:100A300002340534053402340434033404340334FA
:100A400005340534043405340234053403340434E5
:100A500001340234013402340534033403340134E4
:100A600005340534023401340134043404340134CF
:100A700002340134013402340334033403340434C3
:100A800003340134053405340334013403340334AE
:100A900002340234023405340334023405340134A0
:100AA0000434053403340434053403340234043488
:100AB000053401340334013405340234043403347E
:100AC0000234013402340234013402340234043476
:100AD000053401340334013401340434033405345F
:100AE0000434023401340434053404340134013450
:100AF000023405340434043403340234023403343D
:100B0000033401340434023403340434043403342D
:100B10000434043401340134023403340234013423
:100B2000023401340534043405340534023402340B
:100B300002340434053404340334023401340334FD
:100B400003340534033402340334023401340234F0
:100B500001340534013403340534053404340434D9
:100B600003340134053403340134013403340134D3
:100B700003340434053405340534023405340134B7
:100B800001340434013403340234043402340134B3
:100B9000033402340434033401340434023405349D
:100BA0000334013405340334013402340434013491
:100BB0000234013402340334023405340134043481
:100BC000013401340434043402340434053405346B
:100BD0000434023403340534043404340134053459
:100BE0000534053403340534053405340234033444
:100BF000053404340334013402340234033403343E
:02400E00E400CC
:00000001FF
